:060000000A128A11122809
:10000800FE00030EF1000408F2000A08F300831250
:1000180003137F08F4000A128A11A62B0A128A1108
:100028009B2E83120313C001C101BD01BE01B6019D
:10003800B801B70183160313860188018030870051
:100048008312031386018701880106160A128A1192
:10005800E8260A128A118B170B17831603138C16BE
:100068008312031310168F018E010815C001C101F8
:100078004108803AFF0081307F02031D4528003087
:100088004002031C482849284B28662866280A127B
:100098008A11FF260A128A11013083120313C0073E
:1000A8000318C10A0030C1074108803AFF008130B7
:1000B8007F02031D612800304002031C6428652864
:1000C8004B28662883120313C001C1014108803AF6
:1000D800FF0080307F02031D732809304002031C93
:1000E800762877287928DC28DC2883120313BD01B9
:1000F800BE013E08803AFF0080307F02031D86283B
:1001080008303D02031C89288A288C28C628C6285E
:10011800FF3083120313AC004008AD000330031016
:10012800AD0DFF3E031D9328A0302D07AE003D08FE
:100138002E07AF002F0884002C0883138000073097
:10014800AE005230AD005C30AC00AC0BA928AD0B52
:10015800A928AE0BA928B028013083120313BD07C4
:100168000318BE0A0030BE073E08803AFF00803000
:100178007F02031DC12808303D02031CC428C5287E
:100188008C28C628013083120313C0070318C10A3C
:100198000030C1074108803AFF0080307F02031D0C
:1001A800D72809304002031CDA28DB287928DC2804
:1001B8000A128A1147240A128A110A128A114C2536
:1001C8000A128A11831603130C14831203131014D2
:1001D800BB01BC010330BD000030BE00F328450858
:1001E800013A031DF828F928092990300A128A11C2
:1001F800FA250A128A110A128A1147240A128A1148
:1002080083120313C501B8011A294508023A031DD0
:100218000E290F291A290A128A1147240A128A114B
:1002280083120313C501B8011A291A2988158811E0
:100238003D080A128A11BA260A128A118312031378
:100248003E08803AFF0080307F02031D2D290330CD
:100258003D020318302931293C29831203133D0834
:10026800013EBD003E080318013E003EBE00402985
:1002780083120313BD01BE01BB01BC013C08803AD7
:10028800FF0080307F02031D4B2910303B02031C06
:100298004E294F295129A72AA72A0130831203136F
:1002A8003B05B90000303C05BA003A083904031D83
:1002B8005E295F29FC290230A0000030A1003C081B
:1002C800A301A3073B08A201A2070A128A11D62498
:1002D8000A128A11831203132108BA01BA072008E7
:1002E800B901B907C001C1014108803AFF00803057
:1002F8007F02031D812908304002031C84298529B7
:100308008729A029A02983120313081587148710A9
:100318000130C0070318C10A0030C1074108803AFC
:10032800FF0080307F02031D9B2908304002031C18
:100338009E299F298729A02983120313C001C1017F
:100348004108803AFF0080307F02031DAD29083044
:100358004002031CB029B129B329912A912A83129A
:1003680003133D08AC0001300310AC0DFF3E031D24
:10037800B82901302C07AD00A0302D07AE00390890
:10038800AF0002300310AF0DFF3E031DC629031056
:100398002F0D2E07B0003008840083130008B10029
:1003A800400AD8290310B10CFF3E031DD629311885
:1003B800DE29E229831203130815E52983120313A2
:1003C8000811871487100130C0070318C10A0030CC
:1003D800C1074108803AFF0080307F02031DF629DB
:1003E80008304002031CF929FA29B329912A912AD5
:1003F800023083120313A0000030A1003C08A301BF
:10040800A3073B08A201A2070A128A11D6240A12DE
:100418008A11831203132108BA01BA072008B90107
:10042800B907C001C1014108803AFF0080307F024E
:10043800031D202A08304002031C232A242A262AC6
:10044800642A642A831203133908AC0003300310AA
:10045800AC0DFF3E031D2B2AA0302C07AD003D0834
:10046800AE002E072D07AF002F0884008313000865
:10047800B000400A412A0310B00CFF3E031D3F2A7A
:100488003018472A4B2A8312031308154E2A831261
:1004980003130811871487100130C0070318C10A15
:1004A8000030C1074108803AFF0080307F02031DF9
:1004B8005F2A08304002031C622A632A262A642A1B
:1004C80083120313C001C1014108803AFF00803044
:1004D8007F02031D712A08304002031C742A752A02
:1004E800772A912A912A83120313081587148710F3
:1004F8000130C0070318C10A0030C1074108803A1B
:10050800FF0080307F02031D8B2A08304002031C45
:100518008E2A8F2A772A912A912A0130831203136F
:10052800BB070318BC0A0030BC073C08803AFF0030
:1005380080307F02031DA22A10303B02031CA52A2B
:10054800A62A5129A72A831203134608031DAD2A98
:10055800F328C001C1014108803AFF0080307F02C2
:10056800031DB82A08304002031CBB2ABC2ABE2A35
:10057800302B302B83120313BF0108303F02031CBA
:10058800C62AC72AC92A1D2B1D2B4008AC000330D8
:100598000310AC0DFF3E031DCC2A08302C07AD001C
:1005A800A0302D07AE003F082E07AF002F088400AB
:1005B800831300080139B0003008B5003508AC00D5
:1005C80007300310AC0DFF3E031DE52A4008AD00BF
:1005D80003300310AD0DFF3E031DED2AA0302D079B
:1005E800AE003F082E07AF002F0884000008B000B7
:1005F8000310300C2C04B1004008B2000330031083
:10060800B20DFF3E031D032BA0303207B3003F0895
:100618003307B40034088400310880000130AC008E
:100628002C08BF0708303F02031C1B2B1C2BC92AB0
:100638001D2B0130C0070318C10A0030C10741084B
:10064800803AFF0080307F02031D2C2B08304002C7
:10065800031C2F2B302BBE2A83120313C601440818
:1006680038020318382B392B932B0130AC002C0897
:10067800B60708303602031C422B432BF328BF0170
:1006880008303F02031C492B4A2B4C2B8C2B8C2BFC
:100698003808903E840083170008AC00AD01033091
:1006A800FF000310AC0DAD0DFF0B552B2C08003EC1
:1006B800AE002D080318013EFF3EAF001230B00017
:1006C8008830B1002E083007B2002F0803182F0A0F
:1006D8003107B3003F083207840033080318330A90
:1006E800FF000A128A1500200A128A11B4003F0876
:1006F800D83E84003408831380000130AC002C08F5
:10070800BF0708303F02031C8A2B8B2B4C2B8C2BEA
:100718000130AC002C08B807B601F328F3280130E3
:10072800AC002C08B70747303702031C9C2B9D2BC5
:10073800F328B801B701F328F328F328F3280A129D
:100748008A1112288C1EA92BAA2B0C2C8316031392
:100758008C1EAF2BB02B0C2C831203138C121A088F
:10076800F0007008F5007608013A031DBC2BBD2B7C
:10077800C92B75080D3A031DC22BC32BC92B023098
:10078800F0007008C500F601F8017508243A031D49
:10079800CE2BCF2BE42B7608013A031DD42BD52B77
:1007A800E42BF6017808903E840083178001F80155
:1007B800C5010314C50D1812831603138C12E42BFC
:1007C8007608013A031DE92BEA2B012C7508F00085
:1007D8007808903E84007008831780000130F0008C
:1007E8007008F80750307802031CFB2BFC2B012CF7
:1007F8004F30F0007008F800012C75082A3A031DE4
:10080800062C072C0C2CF6010314F60D0C2C0C2CC2
:1008180083120C1C102C112C3A2C831603130C1C5D
:10082800162C172C3A2C831203130C1010108F015E
:100838008E0110140130C2070318C30A0030C30721
:100848004308803AFF0080307F02031D2D2C0530BD
:100858004202031C302C312C3A2C83120313C6019C
:100868000314C60DC201C3013A2C3A2C7408831232
:100878000313FF0073088A0072088400710E830056
:10088800FE0E7E0E090083120313AB010815A801A2
:10089800A9012908803AFF0081307F02031D562CE8
:1008A80000302802031C592C5A2C5C2C762C762CF0
:1008B8000A128A11FF260A128A11013083120313C1
:1008C800A8070318A90A0030A9072908803AFF00D9
:1008D80081307F02031D722C00302802031C752C06
:1008E800762C5C2C83120313AB0109302B02031CFA
:1008F8007E2C7F2C812CB42CB42CAA0108302A021F
:10090800031C872C882C8A2CAA2CAA2CFF30A40024
:100918002B08A50003300310A50DFF3E031D8F2CE7
:10092800A0302507A6002A082607A7002708840064
:100938002408831380000130A4002408AA07083083
:100948002A02031CA82CA92C8A2CAA2C0130A4004A
:100958002408AB0709302B02031CB32CB42C812CC0
:10096800AB01C4010A128A1179260A128A11C32C12
:10097800013083120313A4002408C407C32C831274
:1009880003134408903E840083178008031DCD2C70
:10099800CE2CBC2C1816831603138C168312031343
:1009A8008C12080083120313A601A11FDC2CDD2C76
:1009B800E62CA009A109A00A0319A10AA60103149B
:1009C800A60DE62CA31FE92CEA2CF42CA209A309F6
:1009D800A20A0319A30A0130A4002408A606F42CCD
:1009E800A701A801210820040319FB2CFC2C3A2D8F
:1009F800A5010314A50D0C2D01300310A00DA10DA8
:100A0800FF3E031D012D0130A4002408A5070C2D6D
:100A1800A11F0F2D102D002D122D122D01300310A6
:100A2800A70DA80DFF3E031D132D21082302031D4A
:100A38001F2D20082202031C222D232D2B2D2008D8
:100A4800A2022108031CA303A30227142B2D0130A3
:100A58000310A10CA00CFF3E031D2C2D0130A50294
:100A6800031D372D382D122D3A2D3A2D2608031D3A
:100A78003E2D442DA709A809A70A0319A80A442D41
:100A88002808A101A1072708A001A0074B2D0800ED
:100A98001A3083120313A5004530A4007E30A3004A
:100AA800A30B542DA40B542DA50B542D17308312D2
:100AB8000313A1008B30A2000A128A1128260A12F9
:100AC8008A111A3083120313A5004530A4007E3022
:100AD800A300A30B6D2DA40B6D2DA50B6D2D103050
:100AE80083120313A1008B30A2000A128A11282650
:100AF8000A128A111A3083120313A5004530A40084
:100B08007E30A300A30B862DA40B862DA50B862D66
:100B1800043083120313A1008B30A2000A128A1139
:100B280028260A128A111A3083120313A5004530A9
:100B3800A4007E30A300A30B9F2DA40B9F2DA50B13
:100B48009F2DF23083120313A1008A30A2000A12EB
:100B58008A1128260A128A111A3083120313A50053
:100B68004530A4007E30A300A30BB82DA40BB82DEC
:100B7800A50BB82D080083120313A200C32D8316FA
:100B880003178C18C82DC92DC32DCA2D8312031322
:100B98002208831203178D0083120313200883127F
:100BA80003178C003F3083120313A100210883161A
:100BB80003178C058312031303108B1FE42DE52DF7
:100BC800E62D03148B13831603170C1555308D006F
:100BD800AA308D008C140C1183120313031CF52DFD
:100BE800F62DF92D8B17F92DF92D08008312031313
:100BF800A400A501172E2408840083170008A30069
:100C08002308A00025080A128A11BF250A128A1192
:100C1800013083120313A3002308A4070130A300A3
:100C28002308A507172E2408840083178008031DAE
:100C38001E2E1F2EFF2D202EA00125080A128A1114
:100C4800BF250A128A110800422E831203132208B4
:100C5800FF00210884000A128A1500200A128A114E
:100C68000A128A11D8260A128A1101308312031334
:100C7800A1070318A20A0030A207422E8312031309
:100C88002208FF00210884000A128A1500200A128F
:100C98008A110038031D512E522E292E532E08007A
:100CA80083120313A1006400831603178C185D2EAA
:100CB8005E2E572E5F2E831203132108831203170B
:100CC8008D003F3083120313A000200883160317FA
:100CD8008C050C1403100C18031400300318013091
:100CE800831203170C08782E080083120313A3013C
:100CF8007D2E23080A128A1154260A128A11831299
:100D08000313A2002308903E840022088317800062
:100D18000130A2002208A3072308FF3E903E84006A
:100D28008008031D982E992E7D2E9A2E0800F50115
:100D3800F601F701F801C201C301C401C501C601EA
:100D48008313A0308400E8300A128A11F7260A12A9
:100D58008A11831790308400E0300A128A11F7262E
:100D68000A128A1183010A128A11152883120313A1
:100D7800A00086120613C92ED72E8616D72E061760
:100D8800D72E86160617D72ED72E2008003A031915
:100D9800D72E013A0319C12E033A0319C32E013A7B
:100DA8000319C52ED72E080083120313A000DC2ECA
:100DB80083160313981CE12EE22EDC2EE32E8312F9
:100DC80003132008990008008316031307138717D5
:100DD80024309800903083120313980081308316D2
:100DE80003139900080064008001840A04060319AB
:100DF80000340406F82E83120313871487100800A2
:10100000FF1B0A2883137F1883170008840A03191B
:10101000FF0A08007F087F398A000408840A031940
:10102000FF0A8200FF34FF34FF34FF34FF34FF3403
:10103000FF34FF34FF34FF34FF34FF34FF34FF3418
:10104000FF34FF34FF34FF34FF34FF34FF34FF3408
:10105000FF34FF34FF34FF34FF34FF34FF34FF34F8
:10106000FF34FF34FF34FF34FF34FF34FF34FF34E8
:10107000FF34FF34FF34FF34FF34FF34FF34FF34D8
:10108000FF34FF34FF34FF34FF34FF34FF34FF34C8
:10109000FF34FF34FF34FF34FF34FF34FF34FF34B8
:1010A000FF34FF34FF34FF34FF34FF34FF34FF34A8
:1010B000FF34FF34FF34FF34FF34FF34FF34FF3498
:1010C000FF34FF34FF34FF34FF34FF34FF34FF3488
:1010D000FF34FF34FF34FF34FF34FF34FF34FF3478
:1010E000FF34FF34FF34FF34FF34FF34FF34FF3468
:1010F000FF34FF34FF34FF34FF34FF34FF34FF3458
:10110000FF34FF34FF34FF34FF34F934FF34F93453
:10111000FF34FF34FF34FF34FF34FF34FF34FF3437
:10112000FF34FF34FF348934C33499349934C334E1
:101130009134FF34FF34E734E734E734E334C33425
:10114000E734FF34FF34C334C334F934B934813461
:10115000BF34FF34FF34BF34C334B934BD34C33477
:10116000C734FF34FF34CD34CF348134C734CF3467
:10117000CB34FF34FF349F3481349934F934C33491
:10118000C134FF34FF349934C3349934F934C3344F
:10119000C134FF34FF34CF348134E7349D34E73435
:1011A000CF34FF34FF349934C33499349934C33481
:1011B000C334FF34FF348334C3349F349D34C33489
:1011C0009D34FF34FF34FF34FF34FF34FF34FF34E9
:1011D000FF34FF34FF34FF34FF34FF34FF34FF3477
:1011E000FF34FF34FF34FF34FF34FF34FF34FF3467
:1011F000FF34FF34FF34FF34FF34FF34FF34FF3457
:10120000FF34FF34FF34FF34FF34FF34FF34FF3446
:10121000FF34FF34FF34FF34FF34FF34FF34FF3436
:10122000FF34FF34FF34FF34FF34FF34FF34FF3426
:10123000FF34FF34FF348134E7349934C3349934B4
:101240009934FF34FF34C134C13499349934C134F2
:10125000C134FF34FF34F934C33499349934C3347E
:10126000F934FF34FF349934C13499349934C1349A
:101270009934FF34FF34E1348134B934B9348134E2
:10128000E134FF34FF34E1348134F934B934F934D2
:10129000E134FF34FF348934C33499349934C3348E
:1012A000F934FF34FF3481349934993499349934C2
:1012B0008134FF34FF34E734C334E734E734C334D4
:1012C000E734FF34FF34CF348734C934CF34E334C8
:1012D000CF34FF34FF34E1349934C934D9349934EC
:1012E000E934FF34FF34F934F934C134F934C1340A
:1012F000F934FF34FF34A5349934BD349934BD3406
:10130000A534FF34FF34AD349D349D34B934B93441
:10131000B534FF34FF349934C33499349934C33429
:101320009934FF34FF34C134C134F9349934F93479
:101330009934FF34FF34D934E334C934D934833495
:10134000D934FF34FF34E134C134C9349934993489
:101350009934FF34FF34CF34C33499349934C334CF
:10136000F334FF34FF34E7348134E734A534E73411
:10137000E734FF34FF349934993499349934C334C1
:101380009934FF34FF3499349934C3349934E734B1
:101390009934FF34FF34A934A934A934A934D3349F
:1013A000A934FF34FF34E7349934EB34DB34993417
:1013B000E734FF34FF34E7349934E7349934E734C1
:1013C000DB34FF34FF34F73481349B34D934813437
:1013D000EF34FF34FF34FF34FF34FF34FF34FF3485
:1013E000FF34FF34FF34FF34FF34FF34FF34FF3465
:1013F000FF34FF34FF34FF34FF34FF34FF34FF3455
:10140000FF34FF34FF34FF34FF34FF34FF34FF3444
:10141000FF34FF34FF34FF34FF34FF34FF34FF3434
:10142000FF34FF34FF34FF34FF34FF34FF34FF3424
:10143000FF34FF34FF348134E7349934C3349934B2
:101440009934FF34FF34C134C13499349934C134F0
:10145000C134FF34FF34F934C33499349934C3347C
:10146000F934FF34FF349934C13499349934C13498
:101470009934FF34FF34E1348134B934B9348134E0
:10148000E134FF34FF34E1348134F934B934F934D0
:10149000E134FF34FF348934C33499349934C3348C
:1014A000F934FF34FF3481349934993499349934C0
:1014B0008134FF34FF34E734C334E734E734C334D2
:1014C000E734FF34FF34CF348734C934CF34E334C6
:1014D000CF34FF34FF34E1349934C934D9349934EA
:1014E000E934FF34FF34F934F934C134F934C13408
:1014F000F934FF34FF34A5349934BD349934BD3404
:10150000A534FF34FF34AD349D349D34B934B9343F
:10151000B534FF34FF349934C33499349934C33427
:101520009934FF34FF34C134C134F9349934F93477
:101530009934FF34FF34D934E334C934D934833493
:10154000D934FF34FF34E134C134C9349934993487
:101550009934FF34FF34CF34C33499349934C334CD
:10156000F334FF34FF34E7348134E734A534E7340F
:10157000E734FF34FF349934993499349934C334BF
:101580009934FF34FF3499349934C3349934E734AF
:101590009934FF34FF34A934A934A934A934D3349D
:1015A000A934FF34FF34E7349934EB34DB34993415
:1015B000E734FF34FF34E7349934E7349934E734BF
:1015C000DB34FF34FF34F73481349B34D934813435
:1015D000EF34FF34FF34FF34FF34FF34FF34FF3483
:1015E000FF34FF34413454342B3443344E344D34BF
:1015F00049343D3431342C3432342C3430342C34AE
:1016000030340D340A340034413454342B344334F0
:101610004D34473446343D3431340D340A340034CB
:1016200041345434453430340D340A3400344134B8
:0816300054340D340A34003477
:00000001FF
